:10258F0020202025732020202020202000204C6F89
:10259F006F6B696E6720666F723A202020202020B3
:1025AF000020466F756E6420253264202020202085
:1025BF00202000204D6F64756C6520435055732E9D
:1025CF002E2E2020200020506F6C6C696E672073B8
:1025DF00797374656D20200020666F72206D6F64B3
:1025EF00756C65732E2E2E202000456E61626C690E
:1025FF006E672052656D6F74657300202020202058
:10260F0020202020202020202020200052656361E0
:10261F006C6C696E6720202020202020005072658E
:10262F0076696F757320507265736574200032324E
:10263F0035730033312E3820202000323235000020
:10264F00000021006400323235730000002208FCC4
:10265F000032303600000000600B5400323037007B
:10266F00000000630E1000323232000000004010F4
:10267F00CC00323233204D00005A10CC00323233AE
:10268F00204100005B5EEC00323237000000002377
:10269F006AA4003233302041000066759400323353
:1026AF00302042000067778800323330204300002B
:1026BF0068797C0032333020440000697B7000322F
:1026CF003130000000002000000132343920410079
:1026DF0000240962013234392042000025827A0138
:1026EF00323530204200004200000232363720419E
:1026FF00000012232802323637204200001325F83B
:10270F000232353620413100344650023235362000
:10271F0041320036490C0232353620423100354BFA
:10272F00C80232353620423200374E8402323539F4
:10273F002041000028514002323539204200002943
:10274F00552802323539204300002A5910023235FC
:10275F0039204400002B5CF8023236302041000053
:10276F003060E0023236302042000031620C02321B
:10277F003631204100002C633802323631204200BE
:10278F00002D672002323631204300002E6B0802E5
:10279F00323631204400002F6EF00232363620419F
:1027AF0000003272D802323636204200003373B442
:1027BF00023235302041000041753002323732008D
:1027CF000000005E00000432383120413100380A29
:1027DF002804323831204231003A0B22043238318A
:1027EF00204331003C0C1C04323831204431003E70
:1027FF000D160432383120413200390E10043238B0
:10280F0031204232003B0F0A04323831204332006C
:10281F003D100404323831204432003F10FE0432A0
:10282F003835462041004C11F804323835462042E5
:10283F00004D12F204323835422041004E13EC04A1
:10284F00323835422042004F157C04323931204155
:10285F00000044170C04323931204200004528A0F3
:10286F000432393220410000483A340432393220E0
:10287F00420000493B2E04323932204300004A3CCB
:10288F002804323932204400004B3D2204323936BD
:10289F0020410000643E1C0432393620420000659E
:0E28AF004B0004323531204100005C00000572
:10485C0044034F0000000041038500440353000053
:02486C0000004A
:104BDC00E4FFFE75A70F75B7835384DFF5A775B691
:104BEC001075A70F43842043B30175A90175B10259
:104BFC000FBF00010EEF640F4E70F543B302E5B327
:064C0C0030E4FB758F048B
:014C1200227F
:1051B30075A70F75A406E4F5A5F5A675F4FC75AF00
:1051C3001C75D40F75D70375E10475E2C2F5A722E8
:0D550D00E4F592F593F594F595759104225F
:1054B100758922758E0C758C5D75881075C80422EE
:0C551A00AFA7E4F5A775C80CF5CA8FA771
:015526002262
:1053AD00AFA775A70F75BA1F75BC8475E88075D149
:0653BD000A75BB118FA769
:0153C30022C7
:10508A00E4FE75F00BEEA42451F582E5F03426F522
:10509A0083E493B50703AF06220EEEB439E47FFF2B
:0150AA0022E3
:10475D00E490021FF0A3F0A3F0A3F0E4900221F087
:10476D00A3F0900222E004F07006900221E004F024
:10477D00900221E0B41FEBA3E0B440E6121A27EF3C
:10478D006009E490021FF0A3F0800E900220E00477
:10479D00F0700690021FE004F0D3900220E0942008
:0947AD0090021FE0940340B322C6
:102B4600E4900384F090021F1214DE00000000E4FB
:102B56007F2DFEFDFC90021FE0F8A3E0F9A3E0FA4A
:102B6600A3E0FBC3121476503990021FA3A3A3E07F
:102B76002457F582E43403F583E4F090021FE0FC69
:102B8600A3E0FDA3E0FEA3E0FFE4FAF9F8EF2401D9
:102B9600FFEA3EFEE93DFDE83CFC90021F1214D21E
:102BA60080AD90021F1214DE00000000E47F39FEA3
:102BB600FDFC90021FE0F8A3E0F9A3E0FAA3E0FB16
:102BC600C31214764003022CEC90021FA3A3E0FE6E
:102BD600A3E090265175F00B12150FEE75F00BA4BD
:102BE6002583F583E493900227F090026274FFF048
:102BF600A37425F0A3748FF0E47F0BFEFDFC900216
:102C06001FE0F8A3A3A3E0121419744A2FF974263F
:102C16003EFA90026574FFF0A3EAF0A3E9F07B00A8
:102C26007A007908121A95900262E4F0A37400F013
:102C3600A37408F07BFF7A25799C124C4A900227F0
:102C4600E0FF1251929002231214DE00000000E40D
:102C56007F987E3AFDFC900223E0F8A3E0F9A3E01A
:102C6600FAA3E0FBC312147650547B017A0279284A
:102C7600124EC1EF602190022AE0B41C1A9002297C
:102C8600E0FF900384E02457F582E43403F583EFF4
:102C9600F0900384E004F0900223E0FCA3E0FDA39F
:102CA600E0FEA3E0FFE4FAF9F8EF2401FFEA3EFEB6
:102CB600E93DFDE83CFC9002231214D2809190027B
:102CC6001FE0FCA3E0FDA3E0FEA3E0FFE4FAF9F8B1
:102CD600EF2401FFEA3EFEE93DFDE83CFC90021FC1
:102CE6001214D2022BB290026274FFF0A37425F084
:102CF600A374B0F0900384E0FF900265E4F0A3EFC4
:102D0600F07B007A007908121A9590026274FFF03F
:102D1600A37425F0A374C2F07B007A007908124CE4
:032D26004AD2147A
:012D29002287
:10163B00E4900207F0A3F0F5D9124BDC1251B31270
:10164B00550D1254B11253AD12551A1252C61254F3
:10165B001B124D5012527212557F9003AEE025E0D3
:10166B00FF1254077F2112553443CE0143E680D23B
:10167B00AF12475D90026274FFF0A37425F0A37460
:10168B00E7F07BFF7A2579D5124C4A9002021214AF
:10169B00DE000000007F807E1A7D067C0090020237
:1016AB00E0F8A3E0F9A3E0FAA3E0FBC312148C501B
:1016BB0021900202E0FCA3E0FDA3E0FEA3E02401E5
:1016CB00FFE43EFEE43DFDE43CFC9002021214D22A
:1016DB0080C3122B469002021214DE000000007F22
:1016EB00407E0D7D037C00900202E0F8A3E0F9A39D
:1016FB00E0FAA3E0FBC312148C5021900202E0FC31
:10170B00A3E0FDA3E0FEA3E02401FFE43EFEE43DE5
:10171B00FDE43CFC9002021214D280C31251509093
:10172B00026274FFF0A37426F0A3740AF07BFF7AB5
:10173B002579F9124C4A9002021214DE00000000C7
:10174B007F407E0D7D037C00900202E0F8A3E0F960
:10175B00A3E0FAA3E0FBC312148C5021900202E029
:10176B00FCA3E0FDA3E0FEA3E02401FFE43EFEE4C6
:10177B003DFDE43CFC9002021214D280C312510EC8
:10178B0090026274FFF0A37426F0A3742CF07BFF1D
:10179B007A26791B124C4A124F6BD21443A8204362
:1017AB00E6089003B0E06012E4FF1252AAEF602645
:1017BB009003D0E0FF1255A18019E4FF1252AAEF5B
:1017CB00600612546A1254F07F011252AAEF60069F
:1017DB001254571254F0900207E07002A3E0604DD0
:1017EB00900208E024FFF0900207E034FFF0E07075
:1017FB0002A3E0701F53E6EF90022274FFF0A37474
:10180B0026F0A37442F07BFF7A26793D1241FA430E
:10181B00E6108019301516E4900207F0A3F0900340
:10182B0009A3E0FAA3E0F91215D01254F0124EED11
:10183B00EF607753E6EF12480BEF14603214602A17
:10184B0024FE602124FC601814603214603F24FADB
:10185B00704CC21590020774FDF0A374E8F0803E43
:10186B00900348800D9003438008900303800390FE
:10187B000340A3E0FAA3E0F91215D08021900306F0
:10188B00A3E0FAA3E0F5828A837F01800E90030622
:10189B00A3E0FAA3E0F5828A837FFF1215D443E617
:1018AB0010124EEDEF708C0219B27B017A0279099E
:1018BB00124EC1EF70030219B890020BE024F770BF
:1018CB000302195024FA700302196624FC601124D8
:1018DB00FE6069241270D37D017FFE12559680CA7B
:1018EB007B017A027909900219EBF0A3EAF0A3E9E4
:1018FB00F0900001121332FF12508A900206EFF0A3
:10190B00E075F00BA4244AF9742635F0FA7BFFC07E
:10191B0003C002C001900219E0FBA3E0FAA3E0248C
:10192B0003F9E43AFA900222EBF0A3EAF0A3E9F010
:10193B00D001D002D0031241FA0218B51251501245
:10194B00510E0218B590020BE0640A70030218B531
:10195B007B017A027909124EC180EA7B017A027906
:10196B000990021CEBF0A3EAF0A3E9F0900003123C
:10197B00133264C060030218B590021CE0FBA3E0B5
:10198B00FAA3E0F9900004121332FF9003AFE06F5B
:10199B0060030218B5900005121332FFC3941E406A
:1019AB00030218B51255A11254F00218B5201403F6
:1019BB000217AD90034F12149D7BA07A86790178A4
:1019CB0000C312148C60030217AD1254F090034F36
:0C19DB001214DE00000000C2140217AD60
:031A12000244B3D8
:1044B300C0E0C0F0C083C082C0D075D000C000C0CF
:1044C30001C002C003C004C005C006C007C2CF902C
:1044D3000385E0B40121900353E0FCA3E0FDA3E0D6
:1044E300FEA3E02401FFE43EFEE43DFDE43CFC903A
:1044F30003531214D280099003857401F01255F40A
:10450300D007D006D005D004D003D002D001D0000C
:0B451300D0D0D082D083D0F0D0E032B6
:1050AB00A2AFE433FCC2AF758F0175B7A575B7F12D
:1050BB008F828E83EDF0E4F58FAF04EF24FF92AF78
:0150CB0022C2
:1051D300A2AFE433FDC2AF758F0375B7A575B7F101
:0F51E3008F828E83E4F0F58FAF05EF24FF92AF3C
:0151F200229A
:1048F900900250EEF0A3EFF0A3ECF0A3EDF0EB4A39
:104909006039900250E0FEA3E0FFA3E0FCA3E0F5CC
:10491900828C83E0FD1250ABEB1B70011A9002539D
:10492900E004F07006900252E004F0900251E004B5
:0C493900F070CB900250E004F080C3222C
:0855D200E4900000F0A3F022B8
:104F4500900000E0FEA3E0FF1251D3900000E0FEC8
:104F5500A3E0FF7C007D027B007A021248F9E49011
:064F65000000F0A3F022A1
:0A406200A90590024AEEF0A3EFF06A
:10406C00EE54FEFE900000E0FCA3E0FD7002EE6C4E
:10407C006057ED4C6003124F4590024AE0FEEE543F
:10408C00FEFE7F00900000F0A3EFF090024CEEF0EB
:10409C00A3EFF0A37400F0A37402F07E0290024C24
:1040AC00E475F0011213CB85F082F583E493FD9057
:1040BC00024EE475F0011213CB85F082F583EDF01E
:1040CC00EF1F70011EEF4E70D490024AE0FCA3E08B
:1040DC00FDEC5401FC74022DF58274003CF583E96F
:0140EC00F0E3
:0140ED0022B0
:10499100900243EEF0A3EFF0A3EBF0A3EAF0A3E95A
:1049A100F090024874FFF5F01213CB45F0602690A9
:1049B1000243E475F0011213CBAFF0FE900245E023
:1049C100FBA3E475F0011213CBA9F0FA121319FD40
:0649D10012406280CC22BE
:10486E004202FA00004202A500004202A00000C16E
:05487E000CC10BC10A92
:0A55AC00C20BC20CE49002A4F0222E
:10500000E49002FAF0A3F09002A5F0A3F0A3F090D0
:1050100002A0F0A3F090029BF0A37440F0E4900291
:03502000A3F022D8
:061A1B001255AC02500060
:0D55270075C19043E6019002A27401F022CC
:0D553400AE0712552790029FEEF0021A1BE1
:104FB700E490026AF0A3F0300B02FF22200CFDD22E
:104FC7000B90029DE4F0A37410F09002E8EFF0E478
:044FD700A3F07F01C3
:014FDB0022B3
:104CB700300B0A90029DE07002A3E070037F002290
:104CC70090029EE024FFF090029DE034FFF09002F6
:104CD700E9E0FE04F074EA2EF582E43402F583EF8E
:044CE700F07F012237
:0B558B00300B07C20BD20C1255B622E9
:0A55B600E5C120E5FBC2C4D2C52206
:10427600900264EBF0A3EAF0A3E9F09002A2E070EA
:1042860002FF22900267E0FE6005D3941040037F90
:084296000022124FB7EF604E49
:10429E00E4900269F0900267E0FF900269E0FEC3CD
:1042AE009F5024900264E0FBA3E0FAA3E0F98E8213
:1042BE00758300121332FF124CB7EF7002FF22907B
:1042CE000269E004F080CEE49002A4F012558B90C7
:0E42DE000268E07003200CFD9002A4E0FF22B5
:0342EC007FFF222F
:0E37300090025CEBF0A3EAF0A3E9F0A3EDF049
:10373E00E4FFD39002FBE094009002FAE0648094E0
:10374E008050012253E6FE9002A0E0FEA3E024A7E3
:10375E00F58274023EF583E0FF9002A0E475F0015D
:10376E001213B5FCE5F064404C70069002A0F0A375
:10377E00F090029CE004F0700690029BE004F0E4EE
:10378E00FE90025FE0FDEEC39D5054EEC39F504F7E
:10379E009002A0E0FCA3E024A7F58274023CF5831E
:1037AE00E0FD90025CE0FBA3E0FAA3E0F98E8275E7
:1037BE008300ED1213939002A0E475F0011213B57D
:1037CE00FCE5F064404C70069002A0F0A3F090026D
:1037DE009CE004F0700690029BE004F00E80A2EED6
:1037EE00C39F50299002A0E475F0011213B5FCE5B9
:1037FE00F064404C70069002A0F0A3F090029CE0A2
:10380E0004F0700690029BE004F00E80D29002FB52
:10381E00E024FFF09002FAE034FFF043E60190025C
:0C382E005FE0FEEFC39E50028002AF0678
:01383A00226B
:10537D00D39002FBE094009002FAE06480948040A8
:08538D00047F0180027F002271
:031A1800022F0D8D
:102F0D00C0E0C0F0C083C082C0D075D000C000C08A
:032F1D0006C007E4
:102F2000C209E5C054FE1215AA2FFC082FFC0A2F77
:102F3000C30C2FC30E3075103075122FC9222FD439
:102F4000282FD42A2FC92C2FC92E2FB6C02F6FC2DD
:102F50002F5AE02F5AE200003080C20A9002E8E0C7
:102F6000F5C2C2C5C2C49002E774FFF0023082907D
:102F700002E7E0FFB4FF129002E9E0F5C2C2C5C269
:102F8000C49002E7E4F00230829002E9E0FEEFC371
:102F90009E50179002E7E0FF04F074EA2FF582E4F8
:102FA0003402F583E0F5C2023082D2C49002A4E478
:102FB000F0C20C0230829002A474FDF0D2C5C2C4EB
:102FC0000230829002E774FFF0D20AC2C4C2C1D2BA
:102FD000C5023082E5C2600790029FE0B5C20E9044
:102FE000029AE4F0C2C5C2C4D2C1023082C2C4C2D5
:102FF000C1300A0302307AC2C502308290029AE0E0
:103000007020E5C2F0E0FFC390029CE09F7480F85E
:1030100090029BE0648098500312500090029AE066
:1030200004F090029CE024FFF090029BE034FFF05B
:103030009002A5E0FEA3E024A7F58274023EF5838A
:10304000E5C2F09002A5E475F0011213B5FEE5F0BB
:1030500064404E70069002A5F0A3F090029AE0142E
:10306000F0700E9002FBE004F070069002FAE004AB
:10307000F0D2C1800DC2C4300A08C20AD2C5800293
:10308000D20930091053C17F43C180C2C5C2C4C236
:07309000C1C209C20CC2C05D
:10309700D007D006D000D0D0D082D083D0F0D0E0F7
:0130A70032F6
:051A2700E5C15420FFA1
:011A2C002297
:0855DA00232432303045505308
:0755E20043C14053E6FE2225
:1032360090024DE0FFA3E0FCA3E0FDA3E0FBA3E0CA
:10324600FAA3E0F990025CE519F0E51AA3F0900202
:0632560055E090025EF05D
:10325C00900256EFF0A3ECF0A3EDF0A3EBF0A3EA91
:04326C00F0A3E9F0F2
:1032700090025F7403F0A374E8F0E5C120E5FBD28F
:10328000C1C2C4D2C5E4FF9003CFF030C0FDE5C099
:1032900054FE2440700302333324FE602424E26091
:1032A0000924FE600524E202333BC2C5EF6003023D
:1032B0003341900256E025E044A0F5C27F0302337B
:1032C00041EFB4030A900257E0F5C27F058072EF28
:1032D000B4050B900257A3E0F5C27F068063EF644C
:1032E00006703E90025EE0900259700FE0FBA3E48E
:1032F00075F0011213CBA9F0FA8008E0FBA3E0FA05
:10330000A3E0F9121319F5C290025DE024FFF090DA
:10331000025CE034FFF0E07002A3E070247F0780DD
:1033200020EFB40706D2C47F0980169003CF74053E
:10333000F0800E9003CF7402F080069003CF7401EA
:10334000F0EFB40904C2C080369003CFE0FE6406FB
:103350006012EEB4021690025F74FFF5F01213B51E
:1033600045F06008D2C5E49003CFF0FF9003CFE0B2
:103370006008C2C5D2C4C2C08005C2C002328BE59B
:04338000C120E5FB88
:013384002226
:1033850090024BEFF0A3ECF0A3EDF0A3EBF0A3EA72
:04339500F0A3E9F0C8
:103399009002537403F0A374E8F0E5C120E5FBD271
:1033A900C1C2C4D2C5E4FF9003CFF030C0FDE5C06F
:1033B90054FE24C8700302347624AE607A24CA709D
:1033C9000302347E24FE603824E2600924FE60058D
:1033D90024E2023486C2C5EF700F90024BE025E06B
:1033E90044A0F5C27F0302348CEF64016003023408
:1033F9008C90024BE025E044A1F5C27F0402348C95
:10340900EFB4030A90024CE0F5C27F058075EFB472
:10341900050B90024CA3E0F5C27F068066EFB40667
:1034290006D2C57F01805CEFB404047F028054900A
:1034390003CF7405F0804C90024EE0FBA3E475F0D5
:10344900011213CBA9F0FAE5C2121381900252E0DE
:1034590024FFF0900251E034FFF0E07002A3E07025
:10346900087F09C2C1D2C4801A7F0280169003CF97
:103479007406F0800E9003CF7402F080069003CF9B
:103489007401F0EFB40904C2C080369003CFE0FEA6
:1034990064066012EEB4021690025374FFF5F0123E
:1034A90013B545F06008D2C5E49003CFF0FF90034F
:1034B900CFE06008C2C5D2C4C2C08005C2C0023311
:0634C900B4E5C120E5FBA3
:0134CF0022DA
:1039440090024DEFF0900250EBF0A3EAF0A3E9F0FF
:0839540090024EECF0A3EDF02F
:10395C00751B00543FF51C543F605CC37440951CB0
:10396C00FFE4951BFE900253E0FCA3E0FDC39FEC2B
:10397C009E50068C198D1A80048E198F1A123236AD
:10398C009003CFE060037F022290024FE0251AF0F3
:10399C0090024EE03519F0900255E0700B900251F8
:1039AC00E519851AF01213B5C3900254E0951AF07C
:1039BC00900253E09519F0900253E0F519A3E0F54D
:1039CC001AD3E51A9400E51994004070E51A944056
:1039DC00E519940050131232369003CFE060037F48
:1039EC000222E4F519F51A80D890024DE0FFA3E00D
:1039FC00FCA3E0FDA3E0FBA3E0FAA3E0F990025CDA
:103A0C00E4F074401232529003CFE060037F022244
:103A1C0074C0251AF51A74FF3519F51990024FE088
:103A2C002440F090024EE03400F0900255E070918A
:0E3A3C0090025175F0401213B50239CD7F0093
:013A4A002259
:10534B007B017A027928E4FDFCFF1253C49003CF52
:08535B00E060037F00227F02E5
:015363002227
:104368009002467401F0A37403F0A374C1F0E490C2
:104378000245F0900245E0FFC3940E5025EFFD7C06
:1043880000A3E0FBA3E475F0011213CBA9F0FAE453
:10439800FF1253C4EF60037F0122900245E004F04E
:1043A80080D1E4900245F0900245E0FF9055DA9301
:1043B800FE74C12FF582E43403F583E06E60037F59
:0E43C8000122900245E004F0E0B408DB7F0320
:0143D60022C4
:103B4B00E4900227F012534BEF7002FF229055DAEC
:103B5B00E4939003C1F09055DBE4939003C2F09093
:103B6B0055DCE4939003C3F09055DDE4939003C4CC
:103B7B00F09055DEE4939003C5F09055DFE49390FD
:103B8B0003C6F09055E0E4939003C7F09055E1E441
:103B9B00939003C8F0A37407F0A37480F0A3E4F030
:103BAB00A37402F07B017A0379C190024BE4F0A37A
:103BBB00740EF0E4FDFCFF125331EF60037F002223
:103BCB00124368EF640360037F01227F0E7E007D4A
:103BDB000E7C007B017A027927C3E49F900254F09C
:103BEB0074809E900253F09002557401F0E4FF1222
:103BFB0039449002267401F0900226E0FFC394072B
:103C0B005025EF640360187B017A027927900253E9
:103C1B007480F0A3E4F0A304F0E4FDFC12394490AB
:093C2B000226E004F080D17F03C1
:013C3400226D
:1053C400900251E4F0A304F01233859003CFE0601F
:0753D400037F01227F00228C
:105317009003E1EBF07B017A0379E1900253E4F02B
:0A532700A304F0E4A3F012394422BD
:10504600C007900249E0FFA3E0900251CFF0A3EF22
:10505600F0D0071233859003CFE060037F01227FF3
:02506600002226
:10533100C00790024BE0FFA3E0900253CFF0A3EF30
:0A534100F0E4A3F0D0071239442273
:0E49D70090025DEBF0A3EAF0A3E9F0A3EDF08F
:1049E500E4900262F090025DE0FBA3E0FAA3E0F937
:1049F500A3E0900267F0900261E0900268F0E4FFA6
:104A0500124276EFB4FF0D900262E0FE04F0EEC3B1
:064A1500940340D17E0075
:014A1B002278
:0B4EC100900259EBF0A3EAF0A3E9F027
:104ECC007E007F007D101215D6900259E0FBA3E006
:104EDC00FAA3E0F97D10123730EF7002FF227F0148
:014EEC0022A3
:1054C1000001FF00FF000001010000FF00FF0100DB
:05417700900292EFF040
:10417C00E5682401FFE43567FAA907A37401F0A3ED
:10418C00EAF0A3E9F0900293E0FBA3E0FAA3E0F9D4
:10419C0074019003A86B7008E965827003EA65836B
:1041AC00700D90029304F0A37403F0A37488F09044
:1041BC000293E0FBA3E0FAA3E0F9E569856A838545
:1041CC006B826B7008E965827003EA6583601E90F0
:1041DC000292E0856882856783F0900293A3E0FAEF
:0D41EC00A3E0AE028E67F568900292E0F04D
:0141F90022A3
:10480B0053E6EFE569856A83856B826401700AE57F
:10481B006865827004E56765837003FF802FAB6961
:10482B00056BE56BAA6A7002056A14F9121319FF7E
:10483B0074019003A86B700AE56B65827004E56ADE
:10484B0065837009756901756A03756B8843E6109A
:01485B00223A
:104EED0053E6EFE569856A83856B826401700AE597
:104EFD006865827004E56765837003FF800AAB699E
:0B4F0D00AA6AA96B121319FF43E610FB
:014F18002276
:031A240002361077
:10361000C0E0C083C082C0D075D000C001C002C06D
:0D36200003C005C006C00720DF030236B856
:10362D00E590541FF565656F6019E59030E402D2A1
:10363D0015E565656F90028FF0541F6003756D037E
:10364D0085656FE56D6062156DE56D705CE56E65A8
:10365D006590028FF030E00AE56520E0057F0112EC
:10366D00417790028FE030E10AE56520E1057F02A8
:10367D0012417790028FE030E20AE56520E2057F86
:10368D000412417790028FE030E30AE56520E305EF
:10369D007F0812417790028FE030E40AE56520E45F
:0B36AD00057F1012417785656EC2DFBB
:0636B80020D80330D95DAB
:1036BE0090028FE580F0C2D9C2D8E0FF656C54C08D
:1036CE00604BEFC4131354037E005403FFE56CC428
:1036DE00540CFDED4F24C1F582EE3454F583E49382
:1036EE00FF900290F0A3E566F0EF2566F566E065C3
:1036FE006630E113200E10900290E0B401047F09B1
:0D370E0080027F0A12417790028FE0F56C77
:10371B00D007D006D005D003D002D001D0D0D082B4
:05372B00D083D0E03264
:0F54E10043E60875DA3175DB3175D983D2DE22E7
:1052C6001254E17B017A0379888B698A6A896B8A31
:0B52D600678968E4900387F0025068CD
:10506800900387E0FF30E104C2958002D295EF30CB
:10507800E204C2968002D296EF30E303C29722D2AE
:0250880097226D
:031A2D00024D7FE8
:084D7F00C0E0C083C082C0D077
:104D8700900386E004F0E0B41910A3E030E004B229
:0D4D9700838002D283900386E4F053913FA5
:094DA400D0D0D082D083D0E032DF
:0B559600900387E05FF04DF0025068CA
:103A4B00008040C020A060E0109050D030B070F0EB
:103A5B00088848C828A868E8189858D838B878F85B
:103A6B00048444C424A464E4149454D434B474F48B
:103A7B000C8C4CCC2CAC6CEC1C9C5CDC3CBC7CFCFB
:103A8B00028242C222A262E2129252D232B272F28B
:103A9B000A8A4ACA2AAA6AEA1A9A5ADA3ABA7AFAFB
:103AAB00068646C626A666E6169656D636B676F62B
:103ABB000E8E4ECE2EAE6EEE1E9E5EDE3EBE7EFE9B
:103ACB00018141C121A161E1119151D131B171F15B
:103ADB00098949C929A969E9199959D939B979F9CB
:103AEB00058545C525A565E5159555D535B575F5FB
:103AFB000D8D4DCD2DAD6DED1D9D5DDD3DBD7DFD6B
:103B0B00038343C323A363E3139353D333B373F3FA
:103B1B000B8B4BCB2BAB6BEB1B9B5BDB3BBB7BFB6A
:103B2B00078747C727A767E7179757D737B777F79A
:103B3B000F8F4FCF2FAF6FEF1F9F5FDF3FBF7FFF0A
:011A150022AE
:10540700EF30E104D2818002C281EF30E203D28221
:0454170022C2822209
:10541B007F3812542F7F0612542F7D0EE4FF125546
:04542B005B021A15F1
:10542F00900265EFF0125395EF20E7F9900265E0D7
:04543F00FF024C1309
:1053950075A0FFC2B3D2B4D2B27F14DFFEAFA0EFC7
:0753A500903A4B93FFC2B2E6
:0153AC0022DE
:0555EF007F0102542FB2
:104C1300EF903A4B93F5A07FC87E00EF1F70011E03
:104C2300EF4E70F7C2B3C2B4D2B27E007FC8EF1F9B
:104C330070011EEF4E70F7C2B27E007FC8EF1F7087
:064C4300011EEF4E70F7A8
:014C49002248
:104C8100EF3395E0FE744B2FF582743A3EF583E4E1
:104C910093F5A0C2B4D2B2D2B37FC87E00EF1F7029
:104CA100011EEF4E70F7C2B27E007FC8EF1F700188
:054CB1001EEF4E70F73C
:014CB60022DB
:0C555B009003E2E05FF04DFFF002542FDF
:0E54FF00AE07125395EF20E7F9AF06024C817D
:104CEB00900265EBF0A3EAF0A3E9F0900265E0FB1C
:104CFB00A3E0FAA3E0F91213196017900265A3E47D
:104D0B0075F0011213CBA9F0FA121319FF1254FF0D
:034D1B0080D9221A
:104C4A0090025FEBF0A3EAF0A3E9F01255EFE4FD5E
:104C5A00FF12556790025FE0FBA3E0FAA3E0F912A6
:104C6A004CEBE4FD7F01125567900262E0FBA3E082
:074C7A00FAA3E0F9024CEB84
:0C556700EF75F040A42D2480FF02542FAB
:1050CC00E4900245F0A37422F0A3741DF0A374FFC6
:1050DC00F07B017A027945E4900261F07D0402498B
:0150EC00D7EC
:1050ED00E4900245F0A37422F0A3741EF0A374FFA4
:1050FD00F07B017A027945E4900261F07D0402496A
:01510D00D7CA
:1051F300E4900225F0A37422F0A37401F0A3EFF06E
:105203007B017A027925E4900261F07D040249D79B
:10521300E4900225F0A37422F0A37402F0A3EFF04C
:105223007B017A027925E4900261F07D040249D77B
:10510E00E4900225F0A37422F0A37416F0A374FFAA
:10511E00F07B017A027925E4900261F07D04024968
:01512E00D7A9
:10512F00E4900225F0A37422F0A37417F0A374FF88
:10513F00F07B017A027925E4900261F07D04024947
:01514F00D788
:10515000E490021FF0A37422F0A37414F0A374FF70
:10516000F07B017A02791FE4900261F07D0402492C
:01517000D767
:10517100E49003DAF0A37422F0A3741BF0A374FF8C
:10518100F07B017A0379DAE4900261F07D0402494F
:01519100D746
:10519200900259EFF0A37422F0A3741AF0A374FFE3
:1051A200F07B017A027959E4900261F07D040249B0
:0151B200D725
:104DAD00E4900249F0A37422F0A37404F0A3EFF091
:104DBD00900248E090024DF0A3EDF0A3EBF07B01E3
:0E4DCD007A027949E4900261F07D070249D72D
:104DDB00E4900247F0A37422F0A37405F0A3EFF064
:104DEB00900246E090024BF0A3EDF0A3EBF07B01B9
:0E4DFB007A027947E4900261F07D070249D701
:104E0900E4900234F0A37422F0A37407F0A3EFF046
:104E1900A3EDF0A3EBF0900233E090023AF07B01AE
:0E4E29007A027934E4900261F07D070249D7E5
:104E3700E4900234F0A37422F0A37408F0A3EFF017
:104E4700A3EDF0A3EBF0900233E090023AF07B0180
:0E4E57007A027934E4900261F07D070249D7B7
:1045850020202020496E76616C696420202020203F
:10459500002000202020202020446F6E6520202050
:1045A5002020004E6F7420526573706F6E64696EC3
:1045B500672E2E2E0020202020202000437264200C
:1045C5004E6F7420466F726D6174746400466F722D
:1045D50020507265736574730020202020202020F0
:0445E5002020200072
:105253001255D27E607F027B017A0379AE900248B9
:0F526300E4F0A37406F0124991124F45C21022D5
:103E75009002207404F0E4A3F0A3F09003AE04F0E4
:103E8500A3740FF0E4A3F01252531255D27E607F53
:103E9500017B017A027920900248E4F0A304F01234
:103EA50049917E007F0D7D007B007A00794B1215CC
:103EB500D6E490021FF090021FE0FFC3941E502A23
:103EC50075F00DEFA42408F582E5F03460AF82FEAD
:103ED5007B007A00794B900248E4F0A3740DF01250
:103EE500499190021FE004F080CC7E607F007B0149
:103EF5007A027921900248E4F0A304F01249917EF8
:103F0500617F8E7B017A027922900248E4F0A30456
:073F1500F0124991024F4533
:104D5000906000E493F46007A3E49364046003129A
:104D60003E7578AE7C037D017BFF7A6079027E0020
:0F4D70007F061212F3E49003A9F09003A8F0223B
:1048AC009003A8E0FFC3941E5042A3E0C3941E5093
:1048BC003BEF75F00DA42408F9746035F0FA7BFF1A
:1048CC00784B7C007D007E007F0D1212F39003A9C3
:1048DC00E075F00DA42408F9746035F0FA7BFF78CC
:0D48EC00587C007D007E007F0D1212F3222B
:104A1C00900225EBF0A3EAF0A3E9F09003A9E0C320
:104A2C00941E50301255D29003A9E075F00DA424B9
:104A3C0008F582E5F03460AF82FE900225E0FBA31E
:104A4C00E0FAA3E0F9900248E4F0A3740DF01249E7
:054A5C0091124F4522FC
:0955C0007B007A007958024A1CB4
:104F19003011229003A8E075F00DA42408F97460FB
:104F290035F0FA7BFF784B7C007D007E007F0D1207
:0C4F390012F31255C03010031252532224
:104F6B0090618EE493FFC3941E50099003A9EFF058
:104F7B009003A8F09003A8E0FF1251F31248ACE4A1
:064F8B00FD7FFE025596B9
:104D1E009003A9E09003A8F0E0FF1251F31248AC03
:104D2E00E4FD7FFE1255961255D27E617F8E7B0179
:104D3E007A0379A8900248E4F0A304F01249910294
:024D4E004F45CF
:1052E1007B007A00794B124A1C1248AC9003A9E06A
:0B52F100FF125213E4FD7FFE025596F1
:0B55A1009003A9EFF01248AC024D1E71
:10546A009003A9E004F0E0B41E02E4F01248AC0292
:02547A004D1EC5
:105457009003A9E014F0E0B4FF03741DF01248AC08
:03546700024D1ED5
:0F383B00900226EDF0900225EFF0900227EBF0BF
:10384A00B5070E900226E0FF900228E0B507028035
:10385A002B900227E0FF900225E0C39F5009A3E0C6
:10386A00FEEF9E50028015900227E0FF900225E0AD
:10387A00FED39F401E900228E09E401790025C747F
:10388A00FFF0A37445F0A37496F07BFF7A4579851F
:10389A00023940900225E0FFA3E0FDA3E0FBA3E08C
:1038AA00900233F0124E09900225E0900229F0901E
:1038BA000227E090022AF0900226E0FF900229E017
:1038CA00FED39F505775F00DEEA42408F582E5F05B
:1038DA003460AF8290022EF0FCA3EFF0FD90022A32
:1038EA00E075F00DA42408F582E5F03460FAA982A7
:1038FA007BFF90022BEBF0A3EAF0A3E9F0AE02FF04
:10390A00AA04A905900248E4F0A3740DF0124991A3
:10391A00900229E004F0A3E004F0809B124F4512C4
:10392A0048AC90025C74FFF0A37445F0A37496F05F
:09393A007BFF7A4579981245E9FA
:013943002261
:0F30A800900226EDF0900225EFF0900227EBF05A
:1030B700B5070E900226E0FF900228E0B5070280D0
:1030C7002B900227E0FF900225E0C39F5009A3E061
:1030D700FEEF9E50028015900227E0FF900225E048
:1030E700FED39F401E900228E09E401790025C741A
:1030F700FFF0A37445F0A37496F07BFF7A457985BA
:10310700023232900225E0FFA3E0FDA3E0FBA3E03B
:10311700900233F0124E37900225E0900229F0908A
:103127000227E090022AF0900226E0FF900229E0B1
:10313700D39F400302321BA3E075F00DA42408F5CA
:1031470082E5F03460FAA98290022B74FFF0A3EABB
:10315700F0A3E9F0E4FFFE90022BE0FBA3E0FAA363
:10316700E0F9121319FD74B42FF58274033EF58349
:10317700EDF090022CE475F0011213B50FBF0001BA
:103187000EEF640D4E70D0900229E075F00DA42467
:1031970008F582E5F03460AF8290022EF0FCA3EFD1
:1031A700F0FD90022AE075F00DA42408F582E5F001
:1031B7003460FAA9827BFF90022BEBF0A3EAF0A31D
:1031C700E9F0AE02FFAA04A905900248E4F0A3744F
:1031D7000DF0124991124F45900229E075F00DA4A8
:1031E7002408F582E5F03460AF82FE90022EF0A34A
:1031F700EFF07B017A0379B4900248E4F0A3740DF1
:10320700F0124991124F45900229E004F0A3E0041F
:10321700F002312E1248AC90025C74FFF0A37445A3
:0E322700F0A37496F07BFF7A4579981245E982
:013235002276
:102D2A00E4900248F0900247F0900384E0FF90029A
:102D3A0047E0FEC39F4003022EFD74572EF582E43E
:102D4A003403F583E0FF1251929003AA1214DE00B5
:102D5A000000007B017A027949124EC1EF6010909F
:102D6A00024BE0B41C09900248E004F0022EC6901F
:102D7A0003AAE0FCA3E0FDA3E0FEA3E0FFE4FAF966
:102D8A00F8EF2401FFEA3EFEE93DFDE83CFC900332
:102D9A00AA1214D27F807E847D1E7C009003AAE052
:102DAA00F8A3E0F9A3E0FAA3E0FBC312147670A338
:102DBA00900247E075F00BA4244AF9742635F0FA1C
:102DCA007BFFC00390025CEBF0A37445F0A374A8E8
:102DDA00F0D0031245E9E4900245F0A3F0900245D1
:102DEA00E0FEA3E0FFE4FCFD7B607AEAF9F8D31287
:102DFA0014764010900246E004F070E1900245E03B
:102E0A0004F080D9E4900245F0A3F0900245E0FE78
:102E1A00A3E0FFE4FCFD7B607AEAF9F8D3121476AA
:102E2A004010900246E004F070E1900245E004F0A0
:102E3A0080D9E4900245F0A3F0900245E0FEA3E0B9
:102E4A00FFE4FCFD7B607AEAF9F8D31214764010AD
:102E5A00900246E004F070E1900245E004F080D967
:102E6A00E4900245F0A3F0900245E0FEA3E0FFE4FF
:102E7A00FCFD7B607AEAF9F8D312147640109002CE
:102E8A0046E004F070E1900245E004F080D9E49055
:102E9A000245F0A3F0900245E0FEA3E0FFE4FCFD4A
:102EAA007B607AEAF9F8D31214764010900246E071
:102EBA0004F070E1900245E004F080D9E490024504
:102ECA00F0A3F0900245E0FEA3E0FFE4FCFD7B6086
:102EDA007AEAF9F8D31214764010900246E004F028
:102EEA0070E1900245E004F080D9900247E004F0D6
:102EFA00022D33900384E0FF900248E06F600302E2
:022F0A002D2A6E
:012F0C0022A2
:10222D00E490022CF0A2AF33900231F01255E2127D
:10223D004368900244EFF07F22125534900244E03F
:10224D00640360030225777BFF7A4579BA7F031219
:10225D003D001250CC122D2AE4900226F0900384FA
:10226D00E0FF900226E0FEC39F40030224987457BE
:10227D002EF582E43403F583E0FF90022AF012502C
:10228D008A90022BEFF0E075F00BA4244AF9742626
:10229D0035F0FA7BFF7F03123D0090022BE0FC75B9
:1022AD00F00BA42452F582E5F03426F583E493FE79
:1022BD00740193FDEEFB75F00BECA42454F582E54F
:1022CD00F03426F583E493900248F090022AE0FF63
:1022DD00124DAD9003AA1214DE000000007B017AAE
:1022ED00027934124EC1EF601E900236E0B40A1727
:1022FD007B017A027934900003121332FF90022A87
:10230D00E06F70030224619003AAE0FCA3E0FDA33B
:10231D00E0FEA3E0FFE4FAF9F8EF2401FFEA3EFE48
:10232D00E93DFDE83CFC9003AA1214D27F807E8427
:10233D007D1E7C009003AAE0F8A3E0F9A3E0FAA3C8
:10234D00E0FBC3121476709590022BE075F00BA490
:10235D00244AF9742635F0FA7BFFC00390025CEB3A
:10236D00F0A37445F0A374A8F0D0031245E9E490EE
:10237D000227F0A3F0900227E0FEA3E0FFE4FCFDAE
:10238D007B607AEAF9F8D31214764010900228E0B7
:10239D0004F070E1900227E004F080D9E490022768
:1023AD00F0A3F0900227E0FEA3E0FFE4FCFD7B60CC
:1023BD007AEAF9F8D31214764010900228E004F06E
:1023CD0070E1900227E004F080D9E4900227F0A399
:1023DD00F0900227E0FEA3E0FFE4FCFD7B607AEACB
:1023ED00F9F8D31214764010900228E004F070E151
:1023FD00900227E004F080D9E4900227F0A3F0903A
:10240D000227E0FEA3E0FFE4FCFD7B607AEAF9F829
:10241D00D31214764010900228E004F070E190027F
:10242D0027E004F080D9E4900227F0A3F090022772
:10243D00E0FEA3E0FFE4FCFD7B607AEAF9F8D3123D
:10244D0014764010900228E004F070E1900227E02D
:10245D0004F080D9E4900227F0A3F0900227E0FE6B
:10246D00A3E0FFE4FCFD7B607AEAF9F8D312147661
:10247D004010900228E004F070E1900227E004F093
:10248D0080D9900226E004F002226AC2AF1255E212
:10249D007F2212508A90022BEFF0E0FF75F00BA413
:1024AD002454F582E5F03426F583E493FD90022D56
:1024BD00E4F0A3EDF075F00BEFA42452F582E5F0F6
:1024CD003426F583E493FF74019390022FCFF0A38C
:1024DD00EFF090022BE075F00BA4244AF974263529
:1024ED00F0FA7BFF7F03123D00E4900229F0900289
:1024FD0029E0FFC3941E504B75F00DEFA42408F591
:10250D0082E5F03460AF82FE900232F0FAA3EFF074
:10251D00FB90022DA3E0FFA3E0FCA3E0FDA9037B4C
:10252D00FF90024BE4F0A3740DF012533190023082
:10253D00E0240DF090022FE03400F0900229E00429
:10254D00F080AB7F22125534900231E024FF92AF20
:10255D0090025C74FFF0A37445F0A37496F07BFFBA
:10256D007A4579981245E90250ED90025C74FFF0BE
:10257D00A37445F0A374D2F07BFF7A4579C112455F
:01258D00E964
:01258E00222A
:101EB300A2AFE43390022FF01255E212436890026E
:101EC30042EFF07F22125534900242E06403600334
:101ED3000222157BFF7A4579DE7F02123D00125004
:101EE300CC122D2AE4900225F0900384E0FF9002A7
:101EF30025E0FEC39F400302211A74572EF582E4A6
:101F03003403F583E0FF900229F012508A90022AED
:101F1300EFF0E075F00BA4244AF9742635F0FA7B50
:101F2300FF7F02123D0090022AE0FC75F00BA4240F
:101F330052F582E5F03426F583E493FE740193FDB4
:101F4300EEFB75F00BECA42454F582E5F03426F592
:101F530083E493900246F0900229E0FF124DDB9058
:101F630003AA1214DE000000007B017A0279321208
:101F73004EC1EF601E900234E0B40A177B017A026F
:101F83007932900003121332FF900229E06F70033D
:101F93000220E39003AAE0FCA3E0FDA3E0FEA3E09C
:101FA300FFE4FAF9F8EF2401FFEA3EFEE93DFDE81C
:101FB3003CFC9003AA1214D27F807E847D1E7C0099
:101FC3009003AAE0F8A3E0F9A3E0FAA3E0FBC312AD
:101FD3001476709590022AE075F00BA4244AF974E4
:101FE3002635F0FA7BFFC00390025CEBF0A3744547
:101FF300F0A374A8F0D0031245E9E4900226F0A3FD
:10200300F0900226E0FEA3E0FFE4FCFD7B607AEAA9
:10201300F9F8D31214764010900227E004F070E12F
:10202300900226E004F080D9E4900226F0A3F09019
:102033000226E0FEA3E0FFE4FCFD7B607AEAF9F808
:10204300D31214764010900227E004F070E190025E
:1020530026E004F080D9E4900226F0A3F090022653
:10206300E0FEA3E0FFE4FCFD7B607AEAF9F8D3121B
:1020730014764010900227E004F070E1900226E00D
:1020830004F080D9E4900226F0A3F0900226E0FE4B
:10209300A3E0FFE4FCFD7B607AEAF9F8D31214763F
:1020A3004010900227E004F070E1900226E004F073
:1020B30080D9E4900226F0A3F0900226E0FEA3E08C
:1020C300FFE4FCFD7B607AEAF9F8D3121476401042
:1020D300900227E004F070E1900226E004F080D93A
:1020E300E4900226F0A3F0900226E0FEA3E0FFE4D2
:1020F300FCFD7B507AC3F9F8D3121476401090029A
:1021030027E004F070E1900226E004F080D9900209
:1021130025E004F0021EECC2AF1255E27F221250FA
:102123008A90022AEFF0E0FF75F00BA42454F582A5
:10213300E5F03426F583E493FD90022BE4F0A3ED60
:10214300F075F00BEFA42452F582E5F03426F58305
:10215300E493FF74019390022DCFF0A3EFF090026C
:102163002AE075F00BA4244AF9742635F0FA7BFFB4
:102173007F02123D00E4900228F090022BA3E0FFBF
:10218300A3E0FCA3E0FD7B017A0379B4900249E468
:10219300F0A3740DF012504690022EE0240DF0903F
:1021A300022DE03400F0900228E075F00DA424081D
:1021B300F582E5F03460AF82900230F0A3EFF012C5
:1021C30055D2900230E0FEA3E0FF7B017A0379B49D
:1021D300900248E4F0A3740DF0124991124F459018
:1021E3000228E004F0E0C3941E408F7F221255348E
:1021F30090022FE024FF92AF90025C74FFF0A3746F
:1022030045F0A37496F07BFF7A4579981245E9026D
:1022130050ED90025C74FFF0A37445F0A374D2F008
:092223007BFF7A4579C11245E9FF
:01222C00228F
:1028BD00205072696D6F2056657273696F6E2000BE
:1028CD0020496E697469616C697A696E6720202090
:1028DD000025326420006F6666006F6E0052656DD4
:1028ED0020202020202020446973703A2564004266
:1028FD00617365204368616E6E656C3A20253264A4
:10290D0000456E6200446973005374617473004630
:10291D006F726D617474696E67204361726400003B
:10292D0041726520796F7520737572653F20202087
:10293D00006C6173742F4E4F206E6578742F59455E
:10294D005300202020204E6F2043617264202020F0
:10295D0020002000202020202020446F6E652020A4
:10296D00202020003C2D20432E562E202053616D1B
:10297D0070202D3E003C2D204C61737420204E653F
:10298D007874202D3E00466F726D61742043617224
:10299D00642020202020004D6F64756C6520257308
:1029AD00004669726D7761726520257300507265FE
:1029BD00736574204D6F646966696564002020201D
:1029CD00526573746F72696E67202020002020207D
:1029DD004261636B696E67205570202000202020B6
:1029ED0020436F7079696E67202020200020202001
:1029FD0045786368616E67696E672020202000202E
:102A0D0020204D6F64756C65202573002532642D73
:102A1D002532643A2532642D25326400436F707976
:102A2D002045786368616E676500526573746F72D7
:102A3D00652066726F6D20437264004261636B7531
:102A4D007020746F204361726400204142434445FD
:102A5D00464748494A4B4C4D4E4F50515253545591
:102A6D00565758595A6162636465666768696A6B3F
:102A7D006C6D6E6F707172737475767778797A305C
:102A8D003132333435363738397E21402324255EB3
:102A9D00262A28292D2B3D7C0102FE4F9101030989
:102AAD0054A0010306528E0103034D1E0103405233
:102ABD00E10103435457010348546A00000000002C
:102ACD000102FE5364010309494501034355C90140
:102ADD00034855410103064B670000000000010249
:102AED00FE3C35010309557F01034352FC010348A8
:102AFD0053DB0000000000FF28E3FF28E70004FF80
:102B0D00554E000FFF53F1010FFF55730000FF5499
:102B1D00430100FF46490001FF3F1C0004FF3FC079
:102B2D000007FF44450100FF4E930105FF4E650070
:092B3D0000FF547C0100FF548EDE
:06488300C10E41033F00DD
:10527200E4F524F52390026274FFF0A37428F0A3EE
:0C52820074CDF07BFF7A2879BD024C4A05
:041A0E00E4F52822B1
:1040EE00900225EEF0A3EFF0AF051DEF607A90027F
:1040FE0025E0FEA3E0F5828E83A3A3E493FB740177
:10410E0093FA740293F9E52875F005A4240EF5824E
:10411E00E43403F583EBF0A3EAF0A3E9F090022573
:10412E00E0FEA3E0FFF5828E83E493FCE52875F0B4
:10413E0005A4240CF582E43403F583ECF08F828E13
:10414E0083740193FFE52875F005A4240DF582E430
:10415E003403F583EFF00528900226E02405F09055
:09416E000225E03400F0808022FB
:1047B600AB25AA26A927121319FE75F005A4240C09
:1047C600F582E43403F583E0FFEE75F005A4240DCD
:1047D600F582E43403F583E0FD125567AB25AA267E
:1047E600A92712131975F005A4240EF582E43403E3
:1047F600F583E0F9A3E0FAA3E0900306C9F0A3EA83
:05480600F0A3E9F0221F
:1052FC00AB25AA26A9271213197005E528121381CC
:0B530C00AB25AA26A92774FF02135F3F
:1053DB00AB25AA26A927740112135F121319B5283E
:0653EB0004E4121381220C
:011A160022AD
:104B29007BFF7A1A7916900340EBF0A3EAF0A3E928
:104B3900F0900303EBF0A3EAF0A3E9F0900343EB51
:104B4900F0A3EAF0A3E9F0900348EBF0A3EAF0A39D
:0E4B5900E9F0900306EBF0A3EAF0A3E9F022E6
:10470200900225EBF0A3EAF0A3E9F0124B29900204
:1047120025E0FBA3E0FAA3E0F912153BEA494B605E
:1047220039900225E0FBA3E0FAA3E0F9900003121E
:1047320013E1AAF0F97BFFC003C002C00190022579
:10474200E0FBA3E0FAA3E0F912153B12155B90021D
:0B47520026E475F0051213B580B422B8
:0E42EF00900225EFF0A3EBF0A3EAF0A3E9F0B4
:1042FD0090026274FFF0A37428F0A374DEF0ED2435
:10430D0001FEE433A3F0A3CEF07B017A02792A12E9
:10431D001A95900225E0FFE4FD1255677B017A02A4
:10432D00792A124CEBE4900229F0900226E0FBA3CF
:10433D00E475F0011213CBA9F0FA121319902A5754
:10434D0093FF1254FF900229E004F0E0C3940D4056
:0B435D00D9900225E0FF7D01025567AA
:10528E009003A9E02FF0E0FFB41E04E4F0800AEFD3
:0C529E00B4FF069003A9741DF00248AC98
:104B670090033EE0FE2458F9E4FAFBEE60141213BA
:104B770019700F90033EE02457F8E6600512138181
:104B87008004EF12135F121319FFB44E04744D80A3
:0B4B970005EFB4FF04E4121381D211FB
:014BA20022F0
:0955C90090033EE0600214F022A0
:0D55410090033EE0C3940C5003E004F02200
:084FDC007B01AD07900229F0F2
:104FE400ED12135F121319FFB4FF03E4800A900259
:0C4FF40029E0FEB50705EE14121381221F
:0D554E00EFB40104D20D8002C20DD20F2275
:1053F1007A0379AE7404124FDC9003AEE025E0FF2E
:06540100125407D2102234
:0C5573007A0379AF7410124FDCD21022C2
:011A170022AC
:10494500124F199002FE74FFF0A3743DF0A374C6D4
:10495500F0C20F90030974FFF0A37452F0A37433EF
:10496500F090030674FFF0A37455F0A3744EF09015
:10497500034374FFF0A37452F0A374FCF090034852
:0C49850074FFF0A37453F0A374DBF02265
:10523300124F199002FE74FFF0A37443F0A374D7C6
:10524300F090030974FFF0A3744AF0A374E9F02209
:1054A0007BFF7A2A79CD124702E490033EF0C211C5
:0154B00022D9
:0C557F00124F197BFF7A2A79A50247021F
:103DC6007D027FF312559690026274FFF0A3742869
:103DD600F0A374EAF09003AEE02401FEE43390020F
:103DE60065F0A3CEF07B007A007929121A9590022D
:103DF6006274FFF0A37428F0A374FCF09003AFE0A4
:103E06002401FEE433900265F0A3CEF07B007A0035
:103E1600793A121A95900262E4F0A37400F0A37442
:103E26003AF07B007A007929124C4A7D04E4FF12AD
:103E36005567300F19300D0B12510E7BFF7A297919
:103E46000E801112512F7BFF7A29791280067BFF93
:103E56007A297916124CEB121A0E7E2B7F0A7D03F5
:0F3E66001240EE7525007526007527230247B61A
:104A610090026274FFF0A37429F0A3741CF07B0020
:104A71007A007929121A9590026274FFF0A37429C1
:104A8100F0A3742CF07B007A00793A121A95900207
:104A910062E4F0A37400F0A3743AF07B007A007929
:044AA10029024C4A50
:104AA50090026274FFF0A37429F0A3742DF07B00CB
:104AB5007A007929121A9590026274FFF0A374297D
:104AC500F0A3743EF07B007A00793A121A959002B1
:104AD50062E4F0A37400F0A3743AF07B007A0079E5
:044AE50029024C4A0C
:10502300124AA5124EEDEF60FA53E6EF12480BEF6A
:1050330024FC600724FC70067F01227F002243E6E4
:035043001080E0FA
:10464900EF64017057125023EF6051D20E124A6184
:104659001255E2123B4B900225EFF0701790025C65
:1046690074FFF0A37429F0A3745FF07BFF7A2979B2
:104679004F1245E9900225E0B4031A12222D900247
:104689005C74FFF0A37429F0A3745FF07BFF7A29AF
:0C46990079611245E97F21125534C20EF0
:0146A50022F2
:10544300EFB401089003B07401F08005E49003B059
:04545300F0D2102261
:1043D7009003B0E0900262600C74FFF0A37429F0C0
:1043E700A37471800A74FFF0A37429F0A37482F098
:1043F7007B007A007929121A9590026274FFF0A364
:104407007429F0A37493F07B007A00793A121A9515
:10441700900262E4F0A37400F0A3743AF07B007A90
:10442700007929124C4A121A0E7E2B7F197D02122F
:0E44370040EE7525007526007527240247B655
:1054D1009003A9E0FD7B007A0079587F010242EF39
:105364007D047FF51255961255EF1254D190033EE9
:09537400E02403FD7F01025567EE
:104F91007D087FF91255961255EF9003A8E075F040
:104FA1000DA42408F9746035F0FA7BFFE0FDE4FFFD
:064FB1001242EF0254D190
:1041FA0090021FEBF0A3EAF0A3E9F090026274FFC9
:10420A00F0A37429F0A374A4F090021FE0F9A3E0CC
:10421A00FAA3E0900265C9F0A3EAF0A3E9F07B00F3
:10422A007A007929121A9590026274FFF0A3742910
:10423A00F0A374AEF0900222E0F9A3E0FAA3E090B2
:10424A000265C9F0A3EAF0A3E9F07B007A00793AA3
:10425A00121A95900262E4F0A37400F0A3743AF083
:0C426A007B007A007929124C4AD2142201
:10451E009003DEEBF0A3EAF0A3E9F090026274FFE1
:10452E00F0A37429F0A374A4F09003DEE0F9A3E0E5
:10453E00FAA3E0900265C9F0A3EAF0A3E9F07B00CC
:10454E007A007929121A9590026274FFF0A37429E9
:10455E00F0A374BAF07B007A00793A121A959002A1
:10456E0062E4F0A37400F0A3743AF07B007A007951
:07457E0029124C4AD214225D
:0F54F0009002FEA3E0FAA3E0F91215D002506873
:103F1C00EFB401269002FCE07004A3E0641E700A6A
:103F2C009002FCF0A3741EF0803B9002FDE004F0C4
:103F3C0070339002FCE004F0802BD39002FDE094EF
:103F4C00019002FCE064809480401A900346E0707B
:103F5C0004A3E0641E600E9002FDE024FFF09002CA
:103F6C00FCE034FFF09002FCE0FEA3E0FFC3900302
:103F7C004EE09FEE6480F890034DE064809850050D
:103F8C00EEF0A3EFF0C390034EE09FFF90034DE0E3
:103F9C009EFED3EF940EEE6480948040149002FD4C
:103FAC00E0240EFE9002FCE0340090034DF0A3CE12
:043FBC00F00254F0CB
:103FC000EFB4013290034DE07004A3E0641E700A68
:103FD00090034DF0A3741EF08056900346E07004E9
:103FE000A3E0641E604A90034EE004F07042900328
:103FF0004DE004F0803A9002FCE0FEA3E0FF900365
:104000004DE0FCA3E0FDB5070EECB5060A90034DAC
:10401000EEF0A3EFF08019D3ED9401EC648094806E
:10402000400E90034EE024FFF090034DE034FFF08B
:104030009002FCE0FEA3E0FF90034DE0FCA3E0FD56
:10404000C39FFFEC9EFED3EF940EEE6480948040FD
:104050000EED24F2FEEC34FF9002FCF0A3CEF00251
:0240600054F01A
:104445009002FCA3E0FE90034DA3E0C39EFEEFB4F3
:10445500013C90034BE0FCA3E0FD641E4C700A9008
:10446500034BF0A3741EF08042AF067E00ED2FFFD4
:10447500EE3CFEC3EF941EEE64809480502D9003B5
:104485004CE004F0702590034BE004F0801DD390C0
:10449500034CE0940190034BE064809480400CA3AE
:0E44A500E024FFF090034BE034FFF00254F0EF
:104E6500EF64017028D20E9002FCA3E014FF9003BA
:104E75004DA3E014FD90034BA3E014FB900346E023
:0E4E8500F8A3E014900228F01230A8C20E220A
:1045E900900259EBF0A3EAF0A3E9F0900259E0F93F
:1045F900A3E0FAA3E0900262C9F0A3EAF0A3E9F00C
:104609007B007A007929121A9590025CE0F9A3E0FF
:10461900FAA3E0900262C9F0A3EAF0A3E9F07B00F3
:104629007A00793A121A95900262E4F0A37400F0C4
:10463900A3743AF07B007A007929124C4AD21422E9
:103D0000900246EBF0A3EAF0A3E9F0900245EFF051
:103D1000BF021790026274FFF0A37429F0A374CA63
:103D2000F07B007A007929121A95900245E0B403DD
:103D30001790026274FFF0A37429F0A374DAF07B89
:103D4000007A007929121A95900245E0B404179080
:103D5000026274FFF0A37429F0A374EAF07B007A86
:103D6000007929121A95900245E0B4051790026275
:103D700074FFF0A37429F0A374FAF07B007A007941
:103D800029121A9590026274FFF0A3742AF0A374AA
:103D90000CF0900246E0F9A3E0FAA3E0900265C9B6
:103DA000F0A3EAF0A3E9F07B007A00793A121A95C1
:103DB000900262E4F0A37400F0A3743AF07B007AFE
:063DC000007929024C4AC3
:104E9300EF64017028D20E9002FCA3E014FF90038C
:104EA3004DA3E014FD90034BA3E014FB900346E0F5
:0E4EB300F8A3E014900228F012383BC20E2241
:10547C00EFB4010D125023EF6007D20E121EB3C20F
:02548C000E22EE
:10548E00EFB4010D125023EF6007D20E12222DC27F
:02549E000E22DC
:104AE900124F199002FE74FFF0A3743CF0A37435C1
:104AF900F090030974FFF0A3744BF0A374A3F09032
:104B090002FCE4F0A304F090034DE4F0A304F09058
:104B1900034BE4F0A304F0900346E4F0A304F0226D
:103C35009002FCE0FEA3E0FF90034DE0FAA3E0FB59
:103C4500C39FFFEA9EFE90034BE0FCA3E0FD2FFF20
:103C5500EC3E900346F0A3EFF09002FCE0FEA3E0FB
:103C6500FFC3EB9FEE6480F8EA6480985007E49008
:103C75000346F0A3F090026274FFF0A3742AF0A348
:103C85007419F0A3EEF0A3EFF090034DE0FFA3E06D
:103C9500900267CFF0A3EFF0A3ECF0A3EDF0900353
:103CA50046E0FFA3E090026BCFF0A3EFF07B007A34
:103CB500007929121A9590026274FFF0A3742AF014
:103CC500A37429F07B007A00793A121A9590026262
:103CD500E4F0A37400F0A3743AF07B007A0079292C
:103CE500124C4A121A0E7E2B7F237D051240EE756B
:0B3CF50025017526037527010247B664
:104BA3009002FE74FFF0A37446F0A374A6F0900382
:104BB3000974FFF0A37455F0A3747FF0900343745A
:104BC300FFF0A37452F0A374FCF090034874FFF059
:094BD300A37453F0A374DBF0227B
:1046A60090026274FFF0A3742AF0A37437F07B00C3
:1046B6007A007929121A9590026274FFF0A3742A7F
:1046C600F0A37448F07B007A00793A121A959002AA
:1046D60062E4F0A37400F0A3743AF07B007A0079E8
:1046E60029124C4A121A0E7E2B7F3C7D021240EE96
:0C46F6007525017526037527020247B6E2
:03000000020C00EF
:03000300021A03DB
:03000B00021A06D0
:03001300021A09C5
:03001B00021A0CBA
:03002300021A0FAF
:03002B00021A12A4
:03003300021A1599
:03003B00021A188E
:03004300021A1B83
:03004B00021A1E78
:03005300021A216D
:03005B00021A2462
:03006300021A2757
:03006B00021A2A4C
:03007300021A2D41
:100C0000E4F5D9E5EF7480F5FF7402F5EF787FE441
:100C1000F6D8FD9000007F007E04E4F0A3DFFCDE48
:070C2000FA75816F020C62FE
:104889004103D6004103D8004103D7004103D900B1
:10489900C113C1124203D400004203D200004103F4
:0248A900D1013B
:0655E9009003D6E0FF2252
:1052AA00E4FEEF14600C047010A213E433FEC21380
:0B52BA008007A212E433FEC212AF0610
:0152C50022C6
:0455F40043E8102256
:031A21000234D0BC
:1034D000C0E0C0F0C083C082C0D075D000C000C0C2
:0D34E00001C002C003C004C005C006C00743
:1034ED00C2ED9003D6E09003D8F09003B0E0606297
:1034FD009003D6E5BEF0E0FCE4120DBEE4FBFA79D4
:10350D00087841120CAA9002961214D2E4FFFE7DA7
:10351D00F07C41900296E0F8A3E0F9A3E0FAA3E075
:10352D00FB120D47600C400A9002961214DE41F01A
:10353D000000900296E0FCA3E0FDA3E0FEA3E0FFF7
:10354D00120DF29003D0EFF0D39400404CE014F044
:10355D008047E5BEC4540F9003D6F09003D8E0D356
:10356D009403501D9003D6E0940340159003D2E0D0
:10357D007002A3E0700BD2129003D204F0A374F486
:10358D00F09003D2E07002A3E0600E9003D3E0242C
:10359D00FFF09003D2E034FFF09003D7E09003D911
:1035AD00F0A280E4339003D7F09003D9E0701C9023
:1035BD0003D7E0B401159003D4E07002A3E0700BC3
:1035CD00D2139003D404F0A374F4F09003D4E070FC
:1035DD0002A3E0600E9003D5E024FFF09003D4E049
:0835ED0034FFF0900385E4F0C7
:1035F500D007D006D005D004D003D002D001D0002A
:0B360500D0D0D082D083D0F0D0E032D3
:100CA700020E68EC5D046005E859047003020E5EED
:100CB700120E29580460F6EC4860F2EC7004FDFE51
:100CC700FF22C860DB2481C85009C3986002500620
:100CD700020E659850CAF582E9294B4A7005AB8226
:100CE700020E5475F0007C1A7880C3EF9BEE9AEDE4
:100CF70099400DC3EF9BFFEE9AFEED99FDE842F098
:100D0700DC23ACF0D0E0FFD0E0FED0E0FDAB8220EA
:100D1700E7101BEB60BAEC2CFCEF33FFEE33FEED74
:100D270033FD020E40E803F830E705C0F075F00028
:100D3700EF2FFFEE33FEED33FD40B830E7C280AA58
:100D470074F8CC6480CCC86480C8F582046043C35F
:100D5700EB9FF5F0EA9E42F0E99D42F0E89C45F0F2
:100D670060305018E5825FFFE582F42B5582FB5017
:100D7700210ABA001D09B90019088016E5825BFB34
:100D8700E582F42F5582FF50090EBE00050DBD0008
:100D9700010CC3EB9FF5F0EA9E42F0E99D42F0E8B3
:0D0DA7009C45F06007CC4820E701B3EC222A
:100DB40075F020800E75F010800575F0087D007EBA
:100DC400007F003392D530D503121468EC33401001
:100DD400EF33FFEE33FEED33FDEC33FCD5F0ED22C3
:0E0DE400E5F0247EA2D513CC92E7CDCEFF22FF
:100DF200EDD2E7CD33EC3392D524814006E4FFFEF9
:100E0200FDFC22FCE4CFCECDCC24E0501174FF8057
:100E1200EDC3CC13CCCD13CDCE13CECF13CF0470F4
:070E2200F030D5DE02146878
:101A3000E5192462F582E43402F583E00519229069
:101A4000025F300703900262E475F00112151B0279
:101A500013192000E97F2ED2008018EF540F249034
:101A6000D43440D4FF30040BEF24BFB41A00500329
:101A70002461FFE51A6002151A051DE51D700205B7
:101A80001C30070E90025FE475F00112151BEF0287
:101A900013810219E77403D2078003E4C207F51922
:101AA00090025F121532E4F51AF51CF51DE51A6077
:101AB000077F20121A7380F5751BFFC201C200C296
:101AC00002C203C205C206C208121A3FFF700D30DF
:101AD00007057F00121A84AF1DAE1C22B4255FC219
:101AE000D5C204121A3FFF24D0B40A00501A75F070
:101AF0000A781A30D50508B6FF0106C6A426F620D6
:101B0000D5047002D20380D924CFB41A00EF500458
:101B1000C2E5D204021D76D20180C6D20080C0D2B6
:101B20000280BCD2D580BAD20580B47F20121A734D
:101B30002002077401B51A0040F1121A30FF121A80
:101B400073021AADD208D2068095121A30FB121A0F
:101B500030FA121A30F94A4B700679747A1E7BFFFC
:101B600020022EE51A602A7E008E827583001213F1
:101B70003260060EEE651B70F0C2D5EBC0E0EAC025
:101B8000E0E9C0E0EE121DD7D0E0F9D0E0FAD0E0F5
:101B9000FB121319FF60AAEBC0E0EAC0E0E9C0E065
:101BA000121A73D0E02401F9D0E03400FAD0E0FB3F
:101BB000E51B0460DCD51BD98087D20280A2121DF0
:101BC000B960F7E51B700104120E73A91B600DE5E7
:101BD0001B600914F51B121E61EF60F3EA30E70287
:101BE000F404C3995079EAF4251B0430E701E404B6
:101BF000F51B800D121DB960C1EA051B251B120ED5
:101C000073EA90028EF030E701E4251B04D51B0433
:101C100020050114121DD7E4C0E0121E6190028E4F
:101C2000E0601320E70714F0121A5B802204F0D062
:101C3000E014C0E07F00121A5BE51B6007121A5225
:101C4000151B800B300503121A52D0E0021AADD0DA
:101C5000E00480C4121DB9609EE51B04120E73904F
:101C6000028EEAF0E51B2005026001042404121D27
:011C7000D79C
:101C710074FF04C0E0121E61121A5BE51B2005020D
:101C81006003121A52D0E0B51BE87F45121A659025
:101C9100028EE07F2B30E7047F2DF404C0E0121A9E
:101CA10073D0E075F00A84C0F0121A5CD0E0121A09
:101CB1005C021AAD791080027908C206C208800858
:101CC100D2D5790A8004790AC2D5E51B047002F5E0
:101CD1001BE4FAFDFEFF121A30FC7B0820011312EF
:101CE1001A30FD7B1030000A121A30FE121A30FF32
:101CF1007B20EC3382D592D55013C3E43000069F8C
:101D0100FFE49EFEE42001039DFDE49CFCE4CBF88E
:101D1100C201EC700CCFCECDCCE824F8F870F38082
:101D210017C3EF33FFEE33FEED33FDEC33FCEB3342
:101D3100FB994002FB0FD8E9EB300105F8D0E0C474
:101D410048B201C0E00AEC4D4E4F78207B0070C2D2
:101D5100EAB51B0040BCC0E0121DD9D0F0D0E02094
:101D61000104C4C0E0C4B201C0F0121A5CD0F0D5C5
:101D7100F0EB021AAD1215AA1B4A531CB5581B1BD6
:101D81004C1B17421CB94F1CC1441CC1491B304399
:101D91001CC7551BF4461C54451BBE471E94501BC3
:101DA1001F2D1B232E1B462B1B27231B44201E7D6F
:101DB1002A1ADF4800001B3EE51BB4FF03751B0612
:101DC100121A30FC121A30FD121A30FE121A30FFAC
:101DD100900287020EB0790AA2D5200314300509BA
:101DE100B910020404B9080104A2D5200602500169
:101DF100042002689202B51A005034C0E07F2030FE
:101E010003197F30A20272067205500F121E30C2F2
:101E110002C206C205C2087F30800F300503E9C047
:101E2100E0121A73300503D0E0F9D0E0B51ACC30D6
:101E310005177F30B9100C121A737F583004077FD1
:101E4100788003B90803121A733002057F2D021A34
:101E5100737F202008F87F2B2006F322920280CF87
:101E61007F00B40700500B2487F582E43402F58328
:101E7100E0FF22286E756C6C2900D201121A3030F5
:101E810001F8C201781A30D50108F6021ADF2D5087
:101E9100434958121A302403B405004001E4901E4E
:101EA1008F93121A64743A121A64D203751A0402D7
:021EB1001CB55E
:100E2900E9D2E7C933E833F892D5EDD2E7CD33EC0F
:070E390033FC5002B2D52288
:100E4000EC30E7100FBF000C0EBE00080DBD000413
:100E50000BEB6014A2D5EB13FCED92E7FD2274FFBF
:100E6000FCFDFEFF22E480F8A2D574FF13FC7D8018
:030E7000E480EF2C
:100E7300F920E73624F950037907E4F42402FBE56B
:100E830082158270021583DBF6E024FB501BE960B8
:100E930014E4F0E582158270021583E004F0B40ACD
:0D0EA30008E4F0D9EE7401F00A22C2D52255
:100EB000ED33EC3392D5FA602AB4FF33EDC2E77B11
:100EC000FF60067A0E79D5E4227A0E79DE20D50409
:100ED0007A0E79D9224E614E002B494E46002D499B
:100EE0004E4600E47A08F0A3DAFC7B00740722C0C7
:100EF00083C082ECC0E0EDC0E0EEC0E0EFC0E0EA0D
:100F000075F010A4CAABF075F04DA42BFBE435F0DE
:100F1000FCEA2410FAEB34C5FBEC34D9FCEDC2E753
:100F2000FF75F056A4F42411C5F0F434C58FF0A475
:100F30002AE5F03BE43CF020E7141211E3D0E0FF97
:100F4000D0E0FED0E0FDD0E0FC120CAA8014F40446
:100F50001211E3D0E0FFD0E0FED0E0FDD0E0FC12C3
:100F600010ADD082D083E0FAEDD2E7CD33EC33245C
:100F700082FBE4C3CF33CFCE33CECD33CD33DBF3DF
:100F80007B0775F00A846004F0A31B0AE5F0F0A368
:100F90008FF0740AA4FFACF08EF0740AA42CFEAC9F
:100FA000F050010C8DF0740AA42CFDE435F0F0A390
:050FB000DBDE740722E6
:100FB500020E5EE86480F8E933E83360110460F0FE
:100FC500ED33EC337009E8FCE9FDEAFEEBFF2204A2
:100FD50060DED3EB9FEA9EE99DE8C2E78CF0C2F79D
:100FE50095F0400CE8CCF8E9CDF9EACEFAEBCFFB69
:100FF500120E2985D0F05804700320D5B3E804708B
:10100500075002B2D5020E6892D5EC0460F7E4CC25
:10101500C0E0C398F8603B94186008400DD0E0FB31
:10102500020E40E4FBFAC9FC8028E830E406E4C976
:10103500FBE4CAFCE830E305E4C9CACBFCE8540785
:101045006010F8C3E913F9EA13FAEB13FBEC13FC90
:10105500D8F130F52FC3E49CFCEF9BFFEE9AFEED33
:1010650099FDD0E0FBEF4E4D4C701222DB03020ED2
:1010750065EC2CFCEF33FFEE33FEED33FDED30E791
:10108500EB020E40EF2BFFEE3AFEED39FDD0E0FB13
:1010950050130BBB0003020E68ED13FDEE13FEEFBC
:0810A50013FFEC13FC020E40E6
:1010AD00EC4D6011E8497017ED33EC3304600DE43D
:1010BD00FCFFFEFD22E933E8330470F8020E5E12E8
:1010CD000E2958046009E4CC2481500628500902E9
:1010DD000E68284003020E65C0E0EB4A7044B980EB
:1010ED0006D0E0FB020E54EF4E701CBD8008EBFFE6
:1010FD00EAFEE9FD80EBE98DF0A4FEE5F002119624
:10110D00E9CDF9EAFEEBFFEF89F0A4FCE5F0CE891D
:10111D00F0A42EFFE435F0CD89F0A42DFEE435F0DA
:10112D008067EF4E7005BD80D780C3EF8BF0A4AC08
:10113D00F0EE8BF0A42CFCE435F0F8EF8AF0A42C43
:10114D00E5F038FCE433CB8DF0A42CFCE5F03BF856
:10115D00EE8AF0A42CFCE5F038F8E433CF89F0A446
:10116D002CFCE5F038CF3400CE89F0A42FFFE5F04C
:10117D003EFEE433C98DF0A42EFEE5F039CD8AF0A4
:10118D00A42FFFE5F03EFEE43DFD33D0E0FB50071C
:10119D000BBB000F020E68EC2CFCEF33FFEE33FEA1
:0611AD00ED33FD020E40CF
:1011B3003F8000004120000042C80000447A000044
:1011C300461C400047C35000497424004B189680C6
:1011D3004CBEBC205A0E1BCA6753C21C749DC5AEBD
:1011E300FB60065407601C2323121211EB54386072
:1011F300091211FD12120C1210ADECF8EDF9EEFA12
:10120300EFCB22EB12120C80F1543803241C901103
:10121300B3FE93FC0EEE93FD0EEE930ECE93FF22E0
:100C270002163BE493A3F8E493A34003F68001F292
:100C370008DFF48029E493A3F85407240CC8C333CE
:100C4700C4540F4420C8834004F456800146F6DF9D
:100C5700E4800B010204081020408090485CE47E89
:100C6700019360BCA3FF543F30E509541FFEE49392
:100C7700A360010ECF54C025E060A840B8E493A359
:100C8700FAE493A3F8E493A3C8C582C8CAC583CA84
:100C9700F0A3C8C582C8CAC583CADFE9DEE780BE3C
:0148AB00000C
:10122300E709F608DFFA8046E709F208DFFA803EAD
:1012330088828C83E709F0A3DFFA8032E309F6089A
:10124300DFFA8078E309F208DFFA807088828C8302
:10125300E309F0A3DFFA806489828A83E0A3F608B6
:10126300DFFA805889828A83E0A3F208DFFA804C90
:1012730080D280FA80C680D4806980F28033801067
:1012830080A680EA809A80A880DA80E280CA8033D0
:1012930089828A83ECFAE493A3C8C582C8CCC58348
:1012A300CCF0A3C8C582C8CCC583CCDFE9DEE78018
:1012B3000D89828A83E493A3F608DFF9ECFAA9F097
:1012C300EDFB2289828A83ECFAE0A3C8C582C8CCED
:1012D300C583CCF0A3C8C582C8CCC583CCDFEADE06
:1012E300E880DB89828A83E493A3F208DFF980CC68
:1012F30088F0EF60010E4E60C388F0ED2402B40461
:101303000050B9F582EB2402B4040050AF23234507
:06131300822390127373A7
:10131900BB010689828A83E0225002E722BBFE02D2
:09132900E32289828A83E4932205
:10133200BB010CE58229F582E5833AF583E0225070
:1013420006E92582F8E622BBFE06E92582F8E222BA
:0D135200E58229F582E5833AF583E49322D4
:10135F00BB010989828A83F8E028F022500327F71E
:10136F0022BBFE05F8E328F3228A838982F8E493EF
:02137F00282222
:10138100BB010689828A83F0225002F722BBFE014B
:02139100F32245
:10139300F8BB010DE58229F582E5833AF583E8F090
:1013A300225006E92582C8F622BBFE05E92582C83C
:0213B300F22224
:1013B500C5F0F8A3E028F0C5F0F8E58215827002C3
:0613C5001583E038F02260
:1013CB00A3F8E0C5F025F0F0E582158270021583D5
:0613DB00E0C838F0E82232
:1013E100BB0110E58229F582E5833AF583E0F5F04A
:1013F100A3E0225009E92582F886F008E622BBFE27
:101401000AE92582F8E2F5F008E222E5832AF5836C
:08141100E993F5F0A3E9932231
:10141900E88FF0A4CC8BF0A42CFCE98EF0A42CFC72
:101429008AF0EDA42CFCEA8EF0A4CDA8F08BF0A4F0
:101439002DCC3825F0FDE98FF0A42CCD35F0FCEB4F
:101449008EF0A4FEA9F0EB8FF0A4CFC5F02ECD3914
:0F145900FEE43CFCEAA42DCE35F0FDE43CFC2281
:0E146800C3E49FFFE49EFEE49DFDE49CFC2295
:10147600EB9FF5F0EA9E42F0E99D42F0EC6480C8ED
:0614860064809845F0228D
:10148C00EB9FF5F0EA9E42F0E99D42F0E89C45F0B6
:01149C00222D
:10149D007401FF3395E0FEFDFCA3A3A3E02FFFF045
:1014AD00E582158270021583E03EFEF0E58215821D
:1014BD0070021583E03DFDF0E58215827002158303
:0514CD00E03CFCF022F0
:0C14D200ECF0A3EDF0A3EEF0A3EFF0228D
:1014DE00A8828583F0D083D0821214F51214F512EF
:1014EE0014F51214F5E473E493A3C583C5F0C58314
:1014FE00C8C582C8F0A3C583C5F0C583C8C582C858
:01150E0022BA
:0C150F00A42582F582E5F03583F58322E7
:10151B00F8E0FBA3A3E0F925F0F0E5821582700259
:07152B001583E0FA38F022FD
:09153200EBF0A3EAF0A3E9F022BA
:10153B00BB010789828A830216145005E9F802164B
:10154B0002BBFE05E9F802161D89828A8302162F5B
:10155B00BB011A89828A83D0F0D0E0F8D0E0F9D0B1
:10156B00E0FAD0E0FBE8C0E0C0F00215325016E91B
:10157B00F8D083D082D0E0F9D0E0FAD0E0FBC08283
:10158B00C08302160BBBFE16E9F8D083D082D0E0E5
:0F159B00F9D0E0FAD0E0FBC082C083021626220E
:1015AA00D083D082F8E4937012740193700DA3A3D0
:1015BA0093F8740193F5828883E4737402936860E4
:0615CA00EFA3A3A380DFE4
:0615D0008A838982E473A6
:1019E700EFB40A07740D1219F2740A309811A89906
:1019F700B8130CC2983098FDA899C298B811F63060
:071A070099FDC299F5992237
:1015D600EF4E6012EF60010EEDBB010B89828A832C
:1015E600F0A3DFFCDEFA2289F05007F709DFFCA939
:0C15F600F022BBFEFCF309DFFCA9F02290
:09160200E6FB08E6FA08E6F9220D
:09160B00EBF608EAF608E9F62204
:09161400E0FBA3E0FAA3E0F922D7
:09161D00E2FB08E2FA08E2F922FE
:09162600EBF208EAF208E9F222F5
:0C162F00E493FB740193FA740293F92217
:00000001FF
